 adc

 Timestamp is 4da2a50d (Mon Apr 11 18:51:57 2011)

 Preferred load address is 10000000

 Start         Length     Name                   Class
 0001:00000000 00000004H .CRT$XCA                CODE
 0001:00000004 00000004H .CRT$XCZ                CODE
 0001:00000008 00000004H .CRT$XIA                CODE
 0001:0000000c 00000004H .CRT$XIZ                CODE
 0001:00000010 00000004H .CRT$XPA                CODE
 0001:00000014 00000004H .CRT$XPZ                CODE
 0001:00000018 00000004H .CRT$XTA                CODE
 0001:0000001c 00000004H .CRT$XTZ                CODE
 0001:00000020 000001f0H .rdata                  CODE
 0001:00000210 00000020H .rdata$debug            CODE
 0001:00000230 00001b8cH .text                   CODE
 0001:00001dbc 00000048H .xdata                  CODE
 0001:00001e04 0000003cH .idata$2                CODE
 0001:00001e40 00000014H .idata$3                CODE
 0001:00001e54 00000070H .idata$4                CODE
 0001:00001ec4 0000004cH .idata$6                CODE
 0001:00001f10 00000106H .edata                  CODE
 0002:00000000 00000070H .idata$5                DATA
 0002:00000070 00000008H .data                   DATA
 0002:00000078 00000010H .bss                    DATA
 0003:00000000 00000118H .pdata                  DATA

  Address         Publics by Value              Rva+Base       Lib:Object

 0000:00000000       ___safe_se_handler_table   00000000     <absolute>
 0000:00000000       ___safe_se_handler_count   00000000     <absolute>
 0001:00000000       __xc_a                     10001000     corelib0:crt0init.obj
 0001:00000004       __xc_z                     10001004     corelib0:crt0init.obj
 0001:00000008       __xi_a                     10001008     corelib0:crt0init.obj
 0001:0000000c       __xi_z                     1000100c     corelib0:crt0init.obj
 0001:00000010       __xp_a                     10001010     corelib0:crt0init.obj
 0001:00000014       __xp_z                     10001014     corelib0:crt0init.obj
 0001:00000018       __xt_a                     10001018     corelib0:crt0init.obj
 0001:0000001c       __xt_z                     1000101c     corelib0:crt0init.obj
 0001:0000003c       ??_C@_1DA@PPMNHOKM@?$AAA?$AAD?$AAC?$AA?5?$AA?3?$AA?5?$AAI?$AAn?$AAv?$AAa?$AAl?$AAi?$AAd?$AA?5?$AAI?$AAP?$AAG?$AA?5?$AAC?$AAl?$AAk?$AA?$AN?$AA?6?$AA?$AA@ 1000103c     adc_common_topaz_v1:adc.obj
 0001:0000006c       ??_C@_1CI@OHCJFJPM@?$AAE?$AAR?$AAR?$AAO?$AAR?$AA?3?$AA?5?$AA?$CF?$AAs?$AA?5?$AAl?$AAi?$AAn?$AAe?$AA?5?$AA?$CF?$AAd?$AA?3?$AA?5?$AA?$AA@ 1000106c     adc_common_topaz_v1:adc.obj
 0001:00000098       ??_C@_1KG@JFBLAGKP@?$AAc?$AA?3?$AA?2?$AAw?$AAi?$AAn?$AAc?$AAe?$AAr?$AAo?$AAo?$AAt?$AAs?$AA?2?$AAt?$AAo?$AAp?$AAa?$AAz?$AA?2?$AAw?$AAi?$AAn?$AAc?$AAe?$AA7?$AA0?$AA0?$AA?2?$AAp?$AAl?$AAa@ 10001098     adc_common_topaz_v1:adc.obj
 0001:00000140       ??_C@_1EG@BODOANKG@?$AAE?$AAx?$AAc?$AAe?$AAp?$AAt?$AAi?$AAo?$AAn?$AA?5?$AAi?$AAn?$AA?5?$AAA?$AAD?$AAC?$AA?5?$AAI?$AAO?$AAC?$AAT?$AAL?$AA_?$AAP?$AAO?$AAW?$AAE?$AAR?$AA_?$AAS?$AAE?$AAT@ 10001140     adc_common_topaz_v1:adc.obj
 0001:00000188       ??_C@_1FK@CFOKMKHC@?$AAE?$AAx?$AAc?$AAe?$AAp?$AAt?$AAi?$AAo?$AAn?$AA?5?$AAi?$AAn?$AA?5?$AAD?$AAV?$AAF?$AAC?$AA?5?$AAI?$AAO?$AAC?$AAT?$AAL?$AA_?$AAP?$AAO?$AAW?$AAE?$AAR?$AA_?$AAC?$AAA@ 10001188     adc_common_topaz_v1:adc.obj
 0001:000001e4       ??_C@_1CM@GMJLMKBF@?$AAn?$AAo?$AAt?$AA?5?$AAi?$AAm?$AAp?$AAl?$AAe?$AAm?$AAe?$AAn?$AAt?$AAe?$AAd?$AA?5?$AAy?$AAe?$AAt?$AA?$AN?$AA?6?$AA?$AA@ 100011e4     adc_common_topaz_v1:adc.obj
 0001:00000230       BSPADCCIomuxConfig         10001230 f   adc.obj
 0001:00000248       BSPADCEnableClock          10001248 f   adc.obj
 0001:000002ac       BSPADCGetIPGClock          100012ac f   adc.obj
 0001:000002d4       BSPADCGetHSYNCPolarity     100012d4 f   adc.obj
 0001:000002ec       BSPADCGetHSYNCEnable       100012ec f   adc.obj
 0001:00000304       ADC_Deinit                 10001304 f   adc_common_topaz_v1:adc.obj
 0001:00000370       ADC_Init                   10001370 f   adc_common_topaz_v1:adc.obj
 0001:000005a4       ADC_Open                   100015a4 f   adc_common_topaz_v1:adc.obj
 0001:00000600       ADC_Close                  10001600 f   adc_common_topaz_v1:adc.obj
 0001:00000648       ADC_IOControl              10001648 f   adc_common_topaz_v1:adc.obj
 0001:000014bc       ADC_Read                   100024bc f   adc_common_topaz_v1:adc.obj
 0001:000014e0       ADC_Write                  100024e0 f   adc_common_topaz_v1:adc.obj
 0001:00001504       ADC_Seek                   10002504 f   adc_common_topaz_v1:adc.obj
 0001:00001528       ADC_PowerUp                10002528 f   adc_common_topaz_v1:adc.obj
 0001:00001538       ADC_PowerDown              10002538 f   adc_common_topaz_v1:adc.obj
 0001:00001548       LocalFree                  10002548 f   coredll:COREDLL.dll
 0001:00001558       DeleteCriticalSection      10002558 f   coredll:COREDLL.dll
 0001:00001568       NKDbgPrintfW               10002568 f   coredll:COREDLL.dll
 0001:00001578       Sleep                      10002578 f   coredll:COREDLL.dll
 0001:00001588       InitializeCriticalSection  10002588 f   coredll:COREDLL.dll
 0001:00001598       LocalAlloc                 10002598 f   coredll:COREDLL.dll
 0001:000015a8       GetTickCount               100025a8 f   coredll:COREDLL.dll
 0001:000015b8       LeaveCriticalSection       100025b8 f   coredll:COREDLL.dll
 0001:000015c8       EnterCriticalSection       100025c8 f   coredll:COREDLL.dll
 0001:000015d8       SetLastError               100025d8 f   coredll:COREDLL.dll
 0001:000015e8       MmUnmapIoSpace             100025e8 f   ceddk:CEDDK.dll
 0001:000015f8       MmMapIoSpace               100025f8 f   ceddk:CEDDK.dll
 0001:00001608       DDKClockSetGatingMode      10002608 f   cspddk:CSPDDK.dll
 0001:00001618       DDKClockGetFreq            10002618 f   cspddk:CSPDDK.dll
 0001:00001628       DllMain                    10002628 f   corelib0:dllmain.obj
 0001:00001660       _DllMainCRTStartup         10002660 f   corelib0:pegdmain.obj
 0001:000017f8       __security_init_cookie     100027f8 f   corelib0:seccinit.obj
 0001:00001890       exit                       10002890 f   corelib0:cexit.obj
 0001:000019b4       _exit                      100029b4 f   corelib0:cexit.obj
 0001:000019d4       _cexit                     100029d4 f   corelib0:cexit.obj
 0001:000019ec       _c_exit                    100029ec f   corelib0:cexit.obj
 0001:00001a04       _initterm                  10002a04 f   corelib0:crt0dat.obj
 0001:00001a50       _cinit                     10002a50 f   corelib0:crt0dat.obj
 0001:00001a80       __crt_ExitProcess          10002a80 f   corelib0:exitproc_proxy.obj
 0001:00001aac       GetCurrentProcess          10002aac f i corelib0:exitproc_proxy.obj
 0001:00001ac4       _onexit                    10002ac4 f   corelib0:onexit.obj
 0001:00001ca0       atexit                     10002ca0 f   corelib0:onexit.obj
 0001:00001cf0       __rt_udiv                  10002cf0 f   corelib1:COREDLL.dll
 0001:00001d00       memset                     10002d00 f   corelib1:COREDLL.dll
 0001:00001d10       __C_specific_handler       10002d10 f   corelib1:COREDLL.dll
 0001:00001d20       _XcptFilter                10002d20 f   corelib1:COREDLL.dll
 0001:00001d30       __security_gen_cookie2     10002d30 f   corelib1:COREDLL.dll
 0001:00001d40       free                       10002d40 f   corelib1:COREDLL.dll
 0001:00001d50       realloc                    10002d50 f   corelib1:COREDLL.dll
 0001:00001d60       malloc                     10002d60 f   corelib1:COREDLL.dll
 0001:00001d70       _msize                     10002d70 f   corelib1:COREDLL.dll
 0001:00001d80       CspADCTouchGetBaseRegAddr  10002d80 f   adc_mx25_topaz_v1:adc.obj
 0001:00001d9c       DisableThreadLibraryCalls  10002d9c f   coredll:COREDLL.dll
 0001:00001dac       TerminateProcess           10002dac f   coredll:COREDLL.dll
 0001:00001e04       __IMPORT_DESCRIPTOR_COREDLL 10002e04     coredll:COREDLL.dll
 0001:00001e18       __IMPORT_DESCRIPTOR_CEDDK  10002e18     ceddk:CEDDK.dll
 0001:00001e2c       __IMPORT_DESCRIPTOR_CSPDDK 10002e2c     cspddk:CSPDDK.dll
 0001:00001e40       __NULL_IMPORT_DESCRIPTOR   10002e40     coredll:COREDLL.dll
 0002:00000000       __imp_MmUnmapIoSpace       10004000     ceddk:CEDDK.dll
 0002:00000004       __imp_MmMapIoSpace         10004004     ceddk:CEDDK.dll
 0002:00000008       \177CEDDK_NULL_THUNK_DATA  10004008     ceddk:CEDDK.dll
 0002:0000000c       __imp_Sleep                1000400c     coredll:COREDLL.dll
 0002:00000010       __imp_InitializeCriticalSection 10004010     coredll:COREDLL.dll
 0002:00000014       __imp_LocalAlloc           10004014     coredll:COREDLL.dll
 0002:00000018       __imp_NKDbgPrintfW         10004018     coredll:COREDLL.dll
 0002:0000001c       __imp_LeaveCriticalSection 1000401c     coredll:COREDLL.dll
 0002:00000020       __imp_EnterCriticalSection 10004020     coredll:COREDLL.dll
 0002:00000024       __imp_SetLastError         10004024     coredll:COREDLL.dll
 0002:00000028       __imp_DeleteCriticalSection 10004028     coredll:COREDLL.dll
 0002:0000002c       __imp_GetTickCount         1000402c     coredll:COREDLL.dll
 0002:00000030       __imp_LocalFree            10004030     coredll:COREDLL.dll
 0002:00000034       __imp_TerminateProcess     10004034     coredll:COREDLL.dll
 0002:00000038       __imp_DisableThreadLibraryCalls 10004038     coredll:COREDLL.dll
 0002:0000003c       __imp__msize               1000403c     corelib1:COREDLL.dll
 0002:00000040       __imp___rt_udiv            10004040     corelib1:COREDLL.dll
 0002:00000044       __imp_memset               10004044     corelib1:COREDLL.dll
 0002:00000048       __imp___C_specific_handler 10004048     corelib1:COREDLL.dll
 0002:0000004c       __imp__XcptFilter          1000404c     corelib1:COREDLL.dll
 0002:00000050       __imp___security_gen_cookie2 10004050     corelib1:COREDLL.dll
 0002:00000054       __imp_free                 10004054     corelib1:COREDLL.dll
 0002:00000058       __imp_realloc              10004058     corelib1:COREDLL.dll
 0002:0000005c       __imp_malloc               1000405c     corelib1:COREDLL.dll
 0002:00000060       \177COREDLL_NULL_THUNK_DATA 10004060     coredll:COREDLL.dll
 0002:00000064       __imp_DDKClockGetFreq      10004064     cspddk:CSPDDK.dll
 0002:00000068       __imp_DDKClockSetGatingMode 10004068     cspddk:CSPDDK.dll
 0002:0000006c       \177CSPDDK_NULL_THUNK_DATA 1000406c     cspddk:CSPDDK.dll
 0002:00000070       __security_cookie          10004070     corelib0:seccinit.obj
 0002:00000074       __security_cookie_complement 10004074     corelib0:seccinit.obj
 0002:00000078       _exitflag                  10004078     corelib0:cexit.obj
 0002:0000007c       __onexitend                1000407c     <common>
 0002:00000080       __onexitbegin              10004080     <common>
 0002:00000084       _pRawDllMain               10004084     <common>

 entry point at        0001:00001660

 Static symbols

 0001:000016b0       _DllMainCRTStartupHelper   100026b0 f   corelib0:pegdmain.obj
 0001:000018b0       doexit                     100028b0 f   corelib0:cexit.obj
